:10000000830101308A00D429FC0003088301C70062
:100010000408C8000A08C9008A017008CD007A08DF
:10002000CE007B08CC005908D5007108D4007208B6
:10003000D6007308D8007408D7007508D000760879
:10004000CF007708D1007808D3007908D2000B1DC3
:10005000E2286430F200F301831203133308F10045
:100060003208F0000A128A11D8267408A5006430FC
:10007000F200F3012508F000F1010A128A1112259D
:100080003308F1003208F0007408F002031CF10399
:100090007508F1020A30F2000030F3010A128A11E9
:1000A000D8267408AB006430F10025080A128A11C2
:1000B00006253202F2000A30F1002B080A128A11DA
:1000C00006250A128A117202A70003302202031CBD
:1000D0007C28A2017C282708A00087110716742815
:1000E0002B08A0008715071287169B282508A0005B
:1000F0008715071687129B28220803196B28013AD7
:1001000003197028033A031976289B281830992878
:10011000DB3099288C309928893099284B309928E0
:1001200029309928283099289B3099280830992817
:100130000930C600B6282008F000F63E0318B6289D
:100140000A3E031CB6280030F00200308A00AC30B2
:10015000700703188A0A8200862888288A288C2833
:100160008E28902892289428962898284608860059
:10017000C8288611291CD1288615D12886112A1C49
:10018000D1288615D1288611281CD1288615D1287A
:1001900022080319B928013A0319BE28033A0319A2
:1001A000C32883120313A20A83160D1FE1282F30E0
:1001B0008312C00701300318C1070318C2070318D0
:1001C000C3070B11831203130D1FAF2907148714E4
:1001D0000711A6080319F2282E08AC002F08AD005D
:1001E0000717F7283008AC003108AD0007133B08AB
:1001F0004302031D05293A084202031D0529390857
:100200004102031D052938084002031880294008CF
:10021000F4004108F5004208F6004308F7002D08F5
:10022000F1002C08F000F201F3010A128A11C22732
:10023000E830F4000330F5000030F601F7010A124F
:100240008A113A277008B4007108B5007208B60028
:100250007308B7000130A800AA00A9001030F4000C
:100260002730F500F601F7013408F0003508F100F9
:100270003608F2003708F3000A128A113A270A12E8
:100280008A117308720471047004031955296430CB
:10029000F400F501F601F7013430840083130A12EB
:1002A0008A11B6270A128A118029E830F400033037
:1002B000F500F601F7013408F0003508F1003608C2
:1002C000F2003708F3000A128A113A270A128A113B
:1002D000730872047104700403197F290A30F40052
:1002E000F501F601F7013430840083130A128A11F4
:1002F000B6270A128A1183120313AA018029A801C2
:100300000230831203132602031C8F29E730B40046
:100310000330B500B601B701A801AA01A901003058
:100320004302031D9D2900304202031D9D29003018
:100330004102031D9D2905304002031CA60134081B
:10034000B2003508B3003808C0003908C1003A08C7
:10035000C2003B08C3009C080D1383160D13031342
:1003600083124D08F0004E08FA004C08FB005508B7
:10037000D9005408F1005608F2005808F300570855
:10038000F4005008F5004F08F6005108F700530834
:10039000F8005208F9004808840049088A00470814
:1003A0008300FC0E7C0E0900203084004630E821DA
:1003B00083010730CB00FF30CA004630840047304D
:1003C000EC2183010A128A11682D04068001840A37
:1003D0000406031DE5290034F0000A128A11FC21ED
:1003E0000A128A118000840A040870060319003476
:1003F000ED2983120313CA00CB1B072A4B1B0F2ABC
:100400004B088A004A08CA0A0319CB0A82008313E0
:0E0410004B1883174A08CA0A84000008080027
:1009F6008301C40003178D0083168C130C14831215
:100A06000C0803130800F00000307118700703107B
:100A1600F00D0310F10CF10803190800082DF4017C
:100A2600F5010310F30CF20C031C202D7008F407DB
:100A360071080318710AF5070310F00DF10D72081D
:100A4600730403190034142D8301C500831603179C
:100A56008C18292D83120313450803178D000313E1
:100A6600440803178C0083168C1303108B1B031486
:100A76008B130C1555308D00AA308D008C140C117B
:100A860003188B178301080084008003000AF00016
:100A9600031D5E2D840A8003000AF100031D612DEB
:100AA600840A8003000AF200031D642D840A800371
:100AB600000AF3000034840A0008F100840A0008E2
:100AC600F200840A0008F300003411308316031381
:100AD6009C0025309D0007309F002F308500870140
:100AE6008601FF308312860087133F308700850119
:100AF600053083168100E0308B0010300A128A110F
:100B0600FB24A30011300A128A11FB240A128A114F
:100B1600A4007430F0000130F1008312230870073E
:100B2600AE0071080318710AAF007430F00001308E
:100B3600F10024087007B00071080318710AB100AB
:100B4600A6080319AA2D2F08F1002E08AD2D31088D
:100B5600F1003008F0000310F00DF10D7008F400FC
:100B66007108F500F601F701F001C230F100EB3033
:100B7600F2000B30F3000A128A1112277008B8002F
:100B86007108B9007208BA007308BB00E830BC00EF
:100B9600FD30BD00BE01BF013C30840083130A1244
:100BA6008A1147250A128A117308720471047004A7
:100BB6000319A52E851AA02E851EDF2DA101A10AD7
:100BC6000130A800AA00A900210B222EA230BC00E9
:100BD6005430BD00BE01BF01FF30BC07031103182E
:100BE600013E031DBD07FF3003110318013E031D1F
:0A0BF600BE07FF3003110318013E93
:100C0000031DBF073F083E043D043C04031DEF2DB8
:100C1000851CA30A051DA3032308851A1F2EC400E3
:100C200010300A128A1127250D1210300A128A116B
:100C3000FB240A128A11A3000230A1002308B2008B
:100C4000B301E72D851E222EA230BC005430BD001A
:100C5000BE01BF01FF30BC0703110318013E031D95
:100C6000BD07FF3003110318013E031DBE07FF300F
:100C700003110318013E031DBF073F083E043D0456
:100C80003C0403197B2E2A2EA901A230BC0054304B
:100C9000BD00BE01BF01FF30BC0703110318013EB8
:100CA000031DBD07FF3003110318013E031DBE07DE
:100CB000FF3003110318013E031DBF073F083E0428
:100CC0003D043C04031D4B2E851CA40A051DA403F2
:100CD0002408851A792EC40011300A128A1127259A
:100CE0000D1211300A128A11FB240A128A11A40073
:100CF000A101B200B3012108023A0319442E851E56
:100D00007F2EA230BC005430BD00BE01BF01FF30B9
:100D1000BC0703110318013E031DBD07FF3003117B
:100D20000318013E031DBE07FF3003110318013EE7
:100D3000031DBF073F083E043D043C04031D872EEE
:100D40003408B2003508B300CF2D8101C001C101C4
:100D5000C201C30107158717A6080319B12E871012
:100D6000B22E071083160D178312C00A0319C10A89
:100D70000319C20A0319C30A3B084302031DCA2E02
:100D80003A084202031DCA2E39084102031DCA2E29
:100D900038084002031CB42E871383160D1F8C2DB8
:100DA0008312A60A033026020318A6010D178C2D04
:100DB000F601F401F50172087304031DE22EF0013F
:100DC000F10100341F30F6040310F60AF20DF30DA2
:100DD000031CE52EF30CF20C73087102031DF22EB6
:100DE00072087002031CFA2E7208F0027308031CCA
:100DF000730AF102F40DF50DF60BF61AEA2EF61F42
:100E0000062FF409F40A0319F503F5097408F20032
:100E10007508F300761F0034F009F00A0319F10396
:100E2000F1090034840183120313D901F31F272F22
:100E30000310FF30F007F009031CF107F109031C50
:100E4000F207F209031CF307F3095917D9177708BA
:100E50008039D906F71F3E2F0310FF30F407F4093D
:100E6000031CF507F509031CF607F609031CF70731
:100E7000F7093E2F840183120313D901F801F90108
:100E8000FA01FB01740875047604770403194B2FEB
:100E9000C030D905562FF001F101F201F301F02F16
:100EA0000310F40DF50DF60DF70DD90AF71F502FAD
:100EB000D90A0310F80DF90DFA0DFB0D770873022E
:100EC000031D6C2F76087202031D6C2F75087102CA
:100ED000031D6C2F74087002031C7E2F7814740895
:100EE000F0027508031C750FF1027608031C760FDB
:100EF000F2027708031C770FF3020310F70CF60CCD
:100F0000F50CF40CD90359083F39031D592F591F0B
:100F1000962F0310FF30F007F009031CF107F109C9
:100F2000031CF207F209031CF307F3097008F4002D
:100F30007108F5007208F6007308F7007808F000F1
:100F40007908F1007A08F2007B08F300D91FF02F2E
:100F50000310FF30F007F009031CF107F109031C2F
:100F6000F207F209031CF307F309F02F0008F00061
:100F7000840A0008F100840A0008F200840A0008CC
:100F8000F3003B2F84017008F8007108F900720823
:100F9000FA007308FB00F201F301F001F101031004
:100FA000FB0CFA0CF90CF80C031CE42F7408F00786
:100FB00075080318750FF10776080318760FF20706
:100FC00077080318770FF307780879047A047B040D
:100FD0000319F02F0310F40DF50DF60DF70DCF2FBB
:100FE00084080319003473088000840372088000A9
:100FF0008403710880008403700880000034FF348B
:02400E00323F3F
:00000001FF
